:0400000040EF18F0C5
:08000800046ED8CF05F0E0CF33
:1000100006F00001E9CF0CF0EACF07F0E1CF08F0DD
:10002000E2CF09F0D9CF0AF0DACF0BF0F3CF12F01C
:10003000F4CF13F0FACF14F0F5CF15F0F6CF16F099
:10004000F7CF17F000C00EF001C00FF002C010F0A3
:1000500003C011F0F2AA30EF00F0F2B47BEF0AF027
:100060000EC000F00FC001F010C002F011C003F08C
:100070000CC0E9FF07C0EAFF078E08C0E1FF09C016
:10008000E2FF0AC0D9FF0BC0DAFF12C0F3FF13C0B2
:10009000F4FF14C0FAFF15C0F5FF16C0F6FF17C035
:1000A000F7FF045006C0E0FF05C0D8FF1000BC0FEA
:1000B000F66E000EF7220900F55012000000000055
:1000C0000000005F00000003000300143E143E1413
:1000D000242A7F2A1243330866613649552250008C
:1000E00005030000001C2241000041221C001408EE
:1000F0003E081408083E08080050300000080808B0
:100100000808006060000020100804023E514945C4
:100110003E04027F0000426151494622414949366E
:100120001814127F1027454545393E494949320187
:10013000017109073649494936264949493E003681
:100140003600000056360000081422410014141432
:100150001414004122140802015109063E41595568
:100160005E7E0909097E7F494949363E4141412267
:100170007F4141413E7F494949417F090909013E8B
:100180004141493A7F0808087F00417F41003040E3
:1001900040403F7F081422417F404040407F020C96
:1001A000027F7F0204087F3E4141413E7F090909E9
:1001B000061E2121215E7F09090976264949493217
:1001C00001017F01013F4040403F1F2040201F7F31
:1001D0002010207F41221C2241070870080761512E
:1001E000494543007F4100000204081020000041FF
:1001F0007F0004020102044040404040000102042C
:100200000020545454787F4444443838444444448F
:10021000384444447F385454541804047E05050877
:100220005454543C7F0804047800447D400020402E
:10023000443D007F1028440000417F40007C04784A
:1002400004787C0804047838444444387C1414143A
:1002500008081414147C007C0804044854545420E6
:1002600004043F44443C4040207C1C2040201C3C73
:100270004030403C44281028440C5050503C4464CA
:10028000544C44000836414100007F000041413693
:100290000800020102040200A60FF66E020EF72209
:1002A0000900F550120000000000000000000000EE
:1002B000005F00000000050300050300000020624D
:1002C0003E633E23020000242A7A2F2A1200422590
:1002D0001208245221002056495522584000040398
:1002E0000000000000000000003E224141004141AA
:1002F000223E000000000022147F142200000808A3
:10030000087F0808080050300000000000000808BE
:10031000080808080808606000000000000040208D
:10032000100804020100003E414141413E0000002E
:10033000427F4000000000625151494946000022BE
:1003400041494949360000302824227F2000002FEF
:10035000454545453900003E4949494932000001BB
:100360000161190503000036494949493600002654
:10037000494949493E0000003636000000000000AF
:10038000563600000000000000081422410014143A
:100390001414141414004122140800000000000278
:1003A0000151090906001C2259554D120C00601814
:1003B000161116186000007F494949493600001C93
:1003C000224141412200007F414141221C00007F27
:1003D000494949494100007F090909090100001CF8
:1003E000224149493A00007F080808087F000000C0
:1003F000417F410000000020404040403F00007F1E
:10040000100814224100007F4040404040007F021D
:100410000C300C027F00007F020408107F00001CDB
:10042000224141221C00007F090909090600001C25
:10043000224151225C00007F09091929460000264B
:100440004949494932000101017F01010100003F92
:10045000404040403F00030C3040300C03001F6020
:10046000180618601F0041221408142241000102DE
:100470000478040201000041615149454300000035
:1004800000007F414100002B2C782C2B00004141C3
:100490007F00000000000000020102000000404058
:1004A00040404040400005030000000000000020E4
:1004B000545454780000007F484444380000003809
:1004C00044444428000000384444487F0000003879
:1004D0005454541800000000047E05010000000878
:1004E0005454543C0000007F0804047800000000CD
:1004F000007D00000000002040403D0000000000A2
:100500007F10284400000000017F00000000007CF4
:10051000047804780000007C0804047800000038A7
:10052000444444380000007C1414140800000008FF
:100530001414147C0000007C080404080000004827
:1005400054545424000000043E4444200000003C65
:100550004040207C0000000C3040300C0000001CAB
:100560006018601C0000004428102844000000446B
:10057000582018040000004464544C44000000005B
:100580000008364141000000007F000000004141AA
:1005900036080000000008040408101008000000DD
:1005A000000000000000B40FF66E050EF7220900EF
:1005B000F5501200000000000000000000000000E4
:1005C000000000000000000000000000000000002B
:1005D0000000000000000180018001800180018096
:1005E0000100010001000100000000000180018005
:1005F000000000000000110033006600440000000D
:1006000000000000000000000000000000000000EA
:100610000000000002100210021002101FFC1FFC5C
:1006200004200420042004203FF83FF8084008403C
:10063000084008400000010007E0093011181100CF
:100640000900070001E001100108110819100FE06E
:100650000100000000003802440444084410442013
:1006600044403880011C0222042208221022202249
:10067000401C000000000F001880108011801B003B
:100680000E7C0C101E30332061E040C041E2233666
:100690001E1C0000000008001800300020000000B0
:1006A000000000000000000000000000000000004A
:1006B0000000000000080010003000200060004032
:1006C000004000400040004000400060002000303A
:1006D00000100008100008000C00040006000200D2
:1006E00002000200020002000200060004000C00EA
:1006F000080010000000000000001008081004208E
:10070000024001800180024004200810100800000F
:1007100000000000000000000100010001000100D5
:1007200001003FFC01000100010001000100010087
:1007300000000000000000000000000000000000B9
:1007400000000000000000000000000060006000E9
:100750002000400000000000000000000000000039
:1007600000003FFC0000000000000000000000004E
:100770000000000000000000000000000000000079
:1007800000000000000000000000000060006000A9
:10079000000000000001000200040008001000201A
:1007A000004000800100020004000800100020004A
:1007B00040008000000003C0042008100810181832
:1007C0001008100810081008181808100810042045
:1007D00003C0000000000100030005000900010043
:1007E0000100010001000100010001000100010001
:1007F00007C00000000007E00C10180810080008EF
:1008000000180030006000C00180030006000C00EA
:100810001FF80000000003E00E1018080008000890
:10082000001007E000100008000800080018007021
:100830001FC000000000006000E001A003200620AF
:100840000C201820302020203FFC00200020002019
:1008500000F8000000001FF8100010001000100049
:1008600017E018101008000800080018003000E019
:100870001F800000000000F0038006000C0008004C
:100880001BC01430181810081008180808180C306D
:1008900003C0000000001FFC1008101810100030EA
:1008A00000200060004000C0008000800180010046
:1008B00001000000000003C00C30181810081008D8
:1008C000081007E0081010081008100818180C305D
:1008D00003C00000000003C00C30181010181008EE
:1008E000100818180C2803D800100030006001C050
:1008F0000F000000000000000000000000000000E9
:1009000001800180000000000000000001800180E3
:1009100000000000000000000000000000000000D7
:1009200001800180000000000000000001800180C3
:100930000080010000000006001800600180060031
:100940001800600018000400030000C00020001818
:1009500000060000000000000000000000003FFC56
:100960000000000000003FFC00000000000000004C
:100970000000000000006000180006000180006018
:10098000001800060018002000C003000400180032
:1009900060000000000007E00810100810080808B8
:1009A000003000C001000100000000000180018053
:1009B000000000000000000003C00C30100811A867
:1009C00022642444244424C8137010040C1803E047
:1009D00000000000000001000380028006C0044007
:1009E0000C6008200FE01830101030182008F83E76
:1009F0000000000000003FE0081008080808080890
:100A000008100FE0081808040804080408083FF05C
:100A100000000000000003C80C2818181008300857
:100A20002000200020003000100818180C3003C0EF
:100A30000000000000003FC0083008180808080C3B
:100A4000080408040804080C0808081808303FC007
:100A50000000000000003FF80808080408000840F3
:100A600008400FC0084008400800080408083FF884
:100A70000000000000001FFC040404040400042023
:100A8000042007E0042004200400040004001F00E8
:100A900000000000000003C80C38180810083000DF
:100AA00020002000203E3008100818180C2803C829
:100AB0000000000000007C3E10081008100810081C
:100AC00010081FF8100810081008100810087C3EC5
:100AD00000000000000007C001000100010001004B
:100AE000010001000100010001000100010007C038
:100AF00000000000000000F800200020002000207E
:100B000000200020002000200020102018400F802E
:100B10000000000000003E7C0830086008C009802A
:100B20000B000F00098008C00860083008183E3E1E
:100B30000000000000001F00040004000400040086
:100B400004000400040004000404040404041FFC62
:100B5000000000000000F01E30183838282828282F
:100B60002C682448244826C8228823882108F11E9E
:100B7000000000000000783E1C0814081608130846
:100B80001108118810C8104810681038101878081B
:100B900000000000000003C00C3018181008300CD2
:100BA000200420042004300C100818180C3003C056
:100BB0000000000000001FF0040804040404040402
:100BC000040807F0040004000400040004001F00EF
:100BD00000000000000003C00C3018181008300C92
:100BE000200420042004300C11881A580C3003D241
:100BF000000C000000003FE0081008080808080882
:100C000008100FE0082008300810081808083E3EB9
:100C100000000000000007C808281018100810087D
:100C20000C0003C00030100810081808141013E05E
:100C30000000000000007FFC4104410401000100AD
:100C4000010001000100010001000100010007C0D6
:100C50000000000000007C3E10081008100810087A
:100C60001008100810081008100818180C3003C0DD
:100C70000000000000007C3E100818180810083022
:100C80000C2004200460064002C0028003800100A2
:100C9000000000000000F99F2184218423C4324C0D
:100CA00012481668142814281C380C300810081034
:100CB0000000000000007C7C101018300C6006C0A2
:100CC00003800100038006C00C6018301010787C8F
:100CD0000000000000007C7C1010183008200C6020
:100CE000044006C00380010001000100010007C0AC
:100CF0000000000000001FF810301060004000C02D
:100D0000018001000300060004000C0818083FF8E9
:100D10000000000000F8008000800080008000805B
:100D200000800080008000800080008000800080C3
:100D3000008000F80000000000000000000000003B
:100D400000000000000000000000000000000000A3
:100D5000000000001F00010001000100010001006F
:100D6000010001000100010001000100010001007B
:100D700001001F000180066000000000000000006C
:100D80000000000000000000000000000000000063
:100D90000000000000000000000000000000000053
:100DA0000000000000000000000000000000000043
:100DB0000000FFFF030001000080000000000000B1
:100DC0000000000000000000000000000000000023
:100DD0000000000000000000000000000000000013
:100DE00007C00020002007E00820082008680798B6
:100DF0000000000000001C000400040004000400C7
:100E000005E006100408040804080408061005E0BC
:100E100000000000000000000000000000000000D2
:100E200003E004100800080008000800041003E0B4
:100E300000000000000000E0002000200020002052
:100E400007A008601020102010201020086007B8AC
:100E50000000000000000000000000000000000092
:100E600003C0042008100FF008000800041003E07D
:100E7000000000000000007800880100010001006F
:100E80000FE001000100010001000100010007C0A6
:100E90000000000000000000000000000000000052
:100EA00007D808200820082007C008000FF0100805
:100EB00010080FF000001C000400040004000400EF
:100EC00005E00630041004100410041004101E3C49
:100ED0000000000000000000018001800000000010
:100EE000038000800080008000800080008003E09C
:100EF000000000000000000000C000C00000000072
:100F000001C0004000400040004000400040004060
:100F100010801F00000038000800080008000800CA
:100F200008F8086009800E00090008C008303E7CFF
:100F300000000000000007000100010001000100A6
:100F4000010001000100010001000100010007C0D3
:100F50000000000000000000000000000000000091
:100F6000373818C41084108410841084108439CE4B
:100F70000000000000000000000000000000000071
:100F80001DE00630041004100410041004101E3C70
:100F90000000000000000000000000000000000051
:100FA00003C004200810081008100810042003C013
:100FB0000000000000000000000000000000000031
:100FC0001DE00610040804080408061005E00400EB
:100FD00004001F00000000000000000000000000EE
:100FE00007A00860102010201020086007A0002033
:100FF000002000F8000000000000000000000000D9
:101000000E700290030002000200020002000F8036
:1010100000000000000000000000000000000000D0
:1010200007D0083008100780006008100C100BE093
:1010300000000000000000000200020002000200A8
:101040001FE002000200020002000200011000F096
:101050000000000000000000000000000000000090
:101060001C7004100410041004100410063003DC7B
:101070000000000000000000000000000000000070
:101080003C7808200C60044006C002800380010008
:101090000000000000000000000000000000000050
:1010A000799E11881BD80A500A500E700420042023
:1010B0000000000000000000000000000000000030
:1010C0001E780420024001800240042008103E7C6B
:1010D0000000000000000000000000000000000010
:1010E0001E3C0410063002200360014000C0018055
:1010F00013001E00000000000000000000000000BF
:101100000FF00820084000800100021004100FF0CA
:101110000000000000080010002000200020002037
:10112000002000400020002000200020002000209F
:101130000010000801000100010001000100010091
:101140000100010001000100010001000100010097
:101150000100010010000800040004000400040065
:101160000400020004000400040004000400040061
:101170000800100000000000000000000000000057
:101180003C00430180C2003C000000000000000061
:10119000000000000000000000000000000000004F
:1011A000000000000000000000000000000000003F
:1011B00000000000F76AC40FF66E110EF722090056
:1011C000F550120001000200040008001000200089
:1011D0004000800000010002000400080010002010
:1011E00000400080F76AF40FF66E110EF722090036
:1011F000F55012004A616E00F76A080FF66E120E83
:10120000F7220900F550120046656200F76A1C0FCC
:10121000F66E120EF7220900F55012004D617200B1
:10122000F76A300FF66E120EF7220900F550120021
:1012300041707200F76A440FF66E120EF722090031
:10124000F55012004D617900F76A580FF66E120ED4
:10125000F7220900F55012004A756E00F76A6C0F0C
:10126000F66E120EF7220900F55012004A6C790052
:10127000F76A800FF66E120EF7220900F550120081
:1012800041554700F76A940FF66E120EF7220900D7
:10129000F550120053657000F76AA80FF66E120E33
:1012A000F7220900F55012004F637400F76ABC0F73
:1012B000F66E120EF7220900F55012004E6F7600FE
:1012C000F76AD00FF66E120EF7220900F5501200E1
:1012D00044656300F76AE40FF66E120EF722090008
:1012E000F55012004A414E550000F76AFA0FF66EAB
:1012F000120EF7220900F550120046454252000036
:10130000F76A100FF66E130EF7220900F55012005F
:101310004D4152200000F76A260FF66E130EF72299
:101320000900F55012004150524C0000F76A3C0F82
:10133000F66E130EF7220900F55012004D415920A8
:101340000000F76A520FF66E130EF7220900F550EF
:1013500012004A554E450000F76A680FF66E130EEC
:10136000F7220900F55012004A554C590000F76A5F
:101370007E0FF66E130EF7220900F550120041554C
:1013800047530000F76A940FF66E130EF722090018
:10139000F5501200534550540000F76AAA0FF66E3C
:1013A000130EF7220900F55012004F43544200007B
:1013B000F76AC00FF66E130EF7220900F5501200FF
:1013C0004E4F564D0000F76AD60FF66E130EF722F9
:1013D0000900F5501200444543450000F76AEC0F40
:1013E000F66E130EF7220900F550120053756E20A9
:1013F0000000F76A020FF66E140EF7220900F5508E
:1014000012004D6F6E200000F76A180FF66E140E72
:10141000F7220900F5501200547565200000F76AA4
:101420002E0FF66E140EF7220900F55012005765C4
:1014300064200000F76A440FF66E140EF7220900CC
:10144000F5501200546875200000F76A5A0FF66EC6
:10145000140EF7220900F5501200467269200000B0
:10146000F76A700FF66E140EF7220900F55012009D
:10147000536174200000C26BC2510F0836E3000BA9
:10148000006EBD51800B036E0050031003E093907B
:101490008A8002D093908A90000B006EBF51800B1F
:1014A000036E0050031003E093928A8202D093925D
:1014B0008A92000B006EC151800B036E0050031026
:1014C00003E093948A8402D093948A94D890BC3792
:1014D000BD3793968A86D890BE37BF37D890C0372D
:1014E000C13793968A96C22BC7D792908980000005
:1014F00092908990120094968B865B523AE1D89034
:101500006B35036A57DE0900F5CF03F0B46F03C0F3
:10151000BDF06B51040DF350B76BB66F1B0EB625C3
:10152000E96E000EB721EA6EECCFBFF0ED52EFCFBF
:10153000BEF06B51040DF350BB6BBA6F020EBA25AF
:10154000016E000EBB21036E01501B0FE96E000EF1
:101550000320EA6EECCFC1F0ED52EFCFC0F0B4C083
:10156000BCF089DF6B2B0F0E6B176A2B030E6A170B
:1015700051D06A533AE1D8906B35036A1BDE0900FB
:10158000F5CF03F0B46F03C0BDF06B51040DF35001
:10159000B76BB66F1B0EB625E96E000EB721EA6E6B
:1015A000ECCFBFF0ED52EFCFBEF06B51040DF35016
:1015B000BB6BBA6F020EBA25016E000EBB21036E23
:1015C00001501B0FE96E000E0320EA6EECCFC1F054
:1015D000ED52EFCFC0F0B4C0BCF04DDF6B2B0F0E5F
:1015E0006B176A2B030E6A1715D0D8906B35036AF8
:1015F000E1DD0900F5CF03F0B46F03C0B5F003C01F
:10160000BDF0BC6FBF6BBE6BC16BC06B34DF6A2BB0
:10161000030E6A1794968B96B36BB3510108D8A04A
:10162000B7D0B35103E0010A06E00AD0938AB26B47
:1016300081BAB22B07D09388B26B81B8B22B02D09B
:10164000010EB26FB253D8A485D0696B686B036A80
:10165000B3515C0FE96E000E0320EA6EEF5209E011
:10166000036AB3515E0FE96E000E0320EA6E010EAD
:10167000EF6E036AB3515C0FE96E000E0320EA6E51
:10168000EF6AB25320E1D890B335036A600FE96E78
:10169000000E0320EA6EECCFB5F0ED52EFCFB4F0C0
:1016A000B451D00803E1B55107080DE0D890B33527
:1016B000036A600FE96E000E0320EA6E010EEE264B
:1016C00001E3EF2A46D0B25344E1D890B335036A20
:1016D000600FE96E000E0320EA6EECCFB5F0ED521C
:1016E000EFCFB4F0B451D00834E1B551070831E17F
:1016F000036AB3515E0FE96E000E0320EA6E010E1D
:10170000EF6E036AB351640FE96E000E0320EA6EB8
:10171000EF2A036AB351640FE96E000E0320EA6EEC
:10172000EF500A0809E2036AB351660FE96E000E32
:101730000320EA6E010EEF6ED890B335036A600F96
:10174000E96E000E0320EA6E070EEC6EED52080EF5
:10175000EF6E1CD0036AB3515C0FE96E000E0320DC
:10176000EA6E010EEF6ED890B335036A600FE96E32
:10177000000E0320EA6EEC6AED52EF6A036AB35181
:10178000640FE96E000E0320EA6EEF6AB32B45D7B3
:10179000F29430EF00F054696D65200020536574B9
:1017A00020005965617220004D6F6E7468004461BD
:1017B00074652000204461792000486F7572200014
:1017C0004D696E7574005365636E640093909392D7
:1017D0009394949893968A969396929089909290E7
:1017E00092928992929269EF18F0929689969286D7
:1017F0009294898492946BEF18F0EA6A990EE96EDC
:10180000EF500EE0140E016E006A002EFED7012E7E
:10181000FBD7BF0E006E002EFED700D0EF2EF2D702
:101820001200996B99510F0816E39951040DF3506A
:101830009B6B9A6F1B0E9A25E96E000E9B21EA6E38
:10184000EE52EE52EC6AED52EF6AED52EF6AED5253
:10185000EF6A992BE7D712007BC0EAFF7AC0E9FF55
:10186000A4C0EFFFE92AD8B4EA2AEF6A7A2BD8B4E9
:101870007B2B1200EACFA3F0E9CFA2F09CAF08D0F7
:10188000A28FA2A9A22B9B1F9C1F9B2BD8B49C2B81
:101890009C39F0099E6F9E27E20F9F6F320FA16F58
:1018A0009C510F0B9F279F27A127E90FA06FA0270F
:1018B000A0279B390F0BA027A127A037A137A11F75
:1018C000A1379B510F0BA1279E37070E9D6F0A0E64
:1018D000A007A127FDE39F07A027FDE39E079F2701
:1018E000FDE39D079E27FDE3EA6A9D0EE96E070E64
:1018F000A215A29DED52A21507E1A2B9EE52A2B91E
:1019000003D0200E006E20D0E926000EEA22E95016
:10191000A10803E1EA5201E1A28DEF50006E08E157
:10192000A2BD06D0A2B91BD0A2B702D0200E0BD008
:10193000A2AF06D02D0E006EED50A29DA29F04D046
:10194000A287A299300E0026EACF9CF0E9CF9BF047
:1019500000C0A4F081DF9CC0EAFF9BC0E9FFEE500D
:10196000A2ADD5D71200AD532DE0AC51040DF3500C
:10197000AF6BAE6F1B0EAE25016E000EAF21036E76
:1019800001C0E9FFEA6E1F0ED880AB55B06F036A45
:10199000026A016A010E006EB051B16F07E0D89083
:1019A0000036013602360336B12FF9D70050EF1258
:1019B0000150EC10EF6E0250EC10EF6E0350EC1083
:1019C000EF6E31D0AC51040DF350AF6BAE6F1B0E08
:1019D000AE25016E000EAF21036E01C0E9FFEA6E75
:1019E0001F0ED880AB55B06F036A026A016A010E00
:1019F000006EB051B16F07E0D89000360136023664
:101A00000336B12FF9D7FF0E001A011A021A031A72
:101A10000050EF160150EC14EF6E0250EC14EF6E14
:101A20000350EC14EF6E1200AA6BA2C0A9F0200EB6
:101A3000A95F000EAA5BA935A56FAA35A66FA537C9
:101A4000A637A537A637F80EA517A46BA36BA4532A
:101A5000D8A4A0D0A3510708D8A09CD0A351A525F5
:101A6000A96FA451A621AA6F036EA951AAC0F7FFBE
:101A70004CEC01F0A76F070EA125A86FA7AF08D007
:101A8000A0C0ABF0A8C0ACF0010EAD6F6CDF06D00B
:101A9000A0C0ABF0A8C0ACF0AD6B65DFA807A7ADE8
:101AA00008D0A0C0ABF0A8C0ACF0010EAD6F5BDFFA
:101AB00006D0A0C0ABF0A8C0ACF0AD6B54DFA80757
:101AC000A7AB08D0A0C0ABF0A8C0ACF0010EAD6FC2
:101AD0004ADF06D0A0C0ABF0A8C0ACF0AD6B43DFCE
:101AE000A807A7A908D0A0C0ABF0A8C0ACF0010E11
:101AF000AD6F39DF06D0A0C0ABF0A8C0ACF0AD6BC5
:101B000032DFA807A7A708D0A0C0ABF0A8C0ACF0F0
:101B1000010EAD6F28DF06D0A0C0ABF0A8C0ACF0BE
:101B2000AD6B21DFA807A7A508D0A0C0ABF0A8C067
:101B3000ACF0010EAD6F17DF06D0A0C0ABF0A8C0AF
:101B4000ACF0AD6B10DFA807A7A308D0A0C0ABF026
:101B5000A8C0ACF0010EAD6F06DF06D0A0C0ABF0A0
:101B6000A8C0ACF0AD6BFFDEA807A7A108D0A0C04D
:101B7000ABF0A8C0ACF0010EAD6FF5DE06D0A0C092
:101B8000ABF0A8C0ACF0AD6BEEDEA02BA32BD8B4AD
:101B9000A42B5DD7E3EF0DF09E6B9CC003F09B512F
:101BA0009B2BD8B49C2BE96E03C0EAFFEFCF9DF0CE
:101BB0009D530CE09E5199259F6FA06F9AC0A1F094
:101BC0009DC0A2F031D7080E9E27E7D71200AB5177
:101BD000AD03F3CF01F0F4CF00F0AE03F3500026D5
:101BE000AC51AD03F3500020026E1200AA6BA2C0EC
:101BF000A9F0200EA95F000EAA5BAAC0ACF0A9C094
:101C0000ABF0AE6B050EAD6FE2DF02C0A6F001C017
:101C1000A5F0A46BA36BA453D8A48ED0A351040841
:101C2000D8A08AD0A351A525A96FA451A621AA6F37
:101C3000036EA951AAC0F7FF57EC00F0A76FA1C02F
:101C4000A8F0A7A108D0A0C0ABF0A8C0ACF0010ECE
:101C5000AD6F89DE06D0A0C0ABF0A8C0ACF0AD6B14
:101C600082DEA82BA7A308D0A0C0ABF0A8C0ACF020
:101C7000010EAD6F78DE06D0A0C0ABF0A8C0ACF00E
:101C8000AD6B71DEA82BA7A508D0A0C0ABF0A8C093
:101C9000ACF0010EAD6F67DE06D0A0C0ABF0A8C0FF
:101CA000ACF0AD6B60DEA82BA7A708D0A0C0ABF04E
:101CB000A8C0ACF0010EAD6F56DE06D0A0C0ABF0F0
:101CC000A8C0ACF0AD6B4FDEA82BA7A908D0A0C070
:101CD000ABF0A8C0ACF0010EAD6F45DE06D0A0C0E1
:101CE000ABF0A8C0ACF0AD6B3EDEA82BA7AB08D024
:101CF000A0C0ABF0A8C0ACF0010EAD6F34DE06D0D2
:101D0000A0C0ABF0A8C0ACF0AD6B2DDEA82BA7AD8A
:101D100008D0A0C0ABF0A8C0ACF0010EAD6F23DEC0
:101D200006D0A0C0ABF0A8C0ACF0AD6B1CDEA02B01
:101D3000A32BD8B4A42B6FD7B5EF0EF09E6B9CC02D
:101D400003F09B519B2BD8B49C2BE96E03C0EAFF98
:101D5000EFCF9DF09D530CE09E5199259F6FA06F92
:101D60009AC0A1F09DC0A2F041D7060E9E27E7D7EA
:101D70001200AC6BA2C0ABF0200EAB5F000EAC5BF0
:101D8000AB35A56FAC35A66FA537A637A537A637F7
:101D9000A537A637A537A637E00EA517A46BA36B0A
:101DA000A453D8A438D1A3510F08D8A034D1D890C7
:101DB000A335026EA435036E0250A525A76F03500C
:101DC000A621A86FA8C003F0A751A8C0F7FFD3ECC5
:101DD00002F0A96FA0C0AAF0A9AF08D0AAC0ABF0CA
:101DE000A1C0ACF0010EAD6FBEDD06D0AAC0ABF055
:101DF000A1C0ACF0AD6BB7DDAA2BA9AD08D0AAC0CD
:101E0000ABF0A1C0ACF0010EAD6FADDD06D0AAC045
:101E1000ABF0A1C0ACF0AD6BA6DDAA2BA9AB08D08E
:101E2000AAC0ABF0A1C0ACF0010EAD6F9CDD06D036
:101E3000AAC0ABF0A1C0ACF0AD6B95DDAA2BA9A9EF
:101E400008D0AAC0ABF0A1C0ACF0010EAD6F8BDD25
:101E500006D0AAC0ABF0A1C0ACF0AD6B84DDAA2B5C
:101E6000A9A708D0AAC0ABF0A1C0ACF0010EAD6F1D
:101E70007ADD06D0AAC0ABF0A1C0ACF0AD6B73DDCB
:101E8000AA2BA9A508D0AAC0ABF0A1C0ACF0010E46
:101E9000AD6F69DD06D0AAC0ABF0A1C0ACF0AD6BF0
:101EA00062DDAA2BA9A308D0AAC0ABF0A1C0ACF0F8
:101EB000010EAD6F58DD06D0AAC0ABF0A1C0ACF0EA
:101EC000AD6B51DDAA2BA9A108D0AAC0ABF0A1C06F
:101ED000ACF0010EAD6F47DD06D0AAC0ABF0A1C0DB
:101EE000ACF0AD6B40DDAA2BA72BD8B4A82BA8C0B3
:101EF00003F0A751A8C0F7FFD3EC02F0A96FA9AF78
:101F000008D0AAC0ABF0A1C0ACF0010EAD6F2BDDC4
:101F100006D0AAC0ABF0A1C0ACF0AD6B24DDAA2BFB
:101F2000A9AD08D0AAC0ABF0A1C0ACF0010EAD6F56
:101F30001ADD06D0AAC0ABF0A1C0ACF0AD6B13DDCA
:101F4000AA2BA9AB08D0AAC0ABF0A1C0ACF0010E7F
:101F5000AD6F09DD06D0AAC0ABF0A1C0ACF0AD6B8F
:101F600002DDAA2BA9A908D0AAC0ABF0A1C0ACF091
:101F7000010EAD6FF8DC06D0AAC0ABF0A1C0ACF08A
:101F8000AD6BF1DCAA2BA9A708D0AAC0ABF0A1C009
:101F9000ACF0010EAD6FE7DC06D0AAC0ABF0A1C07B
:101FA000ACF0AD6BE0DCAA2BA9A508D0AAC0ABF0C1
:101FB000A1C0ACF0010EAD6FD6DC06D0AAC0ABF06C
:101FC000A1C0ACF0AD6BCFDCAA2BA9A308D0AAC0EE
:101FD000ABF0A1C0ACF0010EAD6FC5DC06D0AAC05D
:101FE000ABF0A1C0ACF0AD6BBEDCAA2BA9A108D0B0
:101FF000AAC0ABF0A1C0ACF0010EAD6FB4DC06D04E
:10200000AAC0ABF0A1C0ACF0AD6BADDCA12BA32B93
:10201000D8B4A42BC5D624EF10F09E6B9CC003F05F
:102020009B519B2BD8B49C2BE96E03C0EAFFEFCFEA
:102030009DF09D530CE09E5199259F6FA06F9AC013
:10204000A1F09DC0A2F095D6100E9E27E7D783EF92
:1020500010F08E6B8D6B11EC0CF08E533AE18D51BC
:10206000C70837E37B6B8F0E7A6F020EE96E8EC066
:102070009CF08DC09BF03AEC0CF0996B9A6B9C6BCA
:102080008F0E9B6F89DD8EC0ACF08DC0ABF0AE6B58
:102090001F0EAD6F9CDD02C09AF001C099F07B6B02
:1020A0008F0E7A6F010EE96E02C09CF001C09BF0AA
:1020B0003AEC0CF0996B080E9A6F9C6B8F0E9B6F2D
:1020C0003DDE020E996FFDEC0BF08D2BD8B48E2BFC
:1020D000C4D78E6B8D6B11EC0CF08E531CE18D51BF
:1020E0001D0819E37B6B8F0E7A6F040EE96E8EC0AC
:1020F0009CF08DC09BF03AEC0CF0996B9A6B9C6B4A
:102100008F0E9B6F8AD7320E996FFDEC0BF08D2BE3
:10211000D8B48E2BE2D711EC0CF08B6B8B511F08CF
:1021200013E38C6B8C510F080DE38BC0ABF08CC0AC
:10213000ACF0010EAD6F17DC020E996FFDEC0BF0E9
:102140008C2BF0D78B2BEAD78B6B8B511F0812E3AC
:102150008C6B8C510F080CE38BC0ABF08CC0ACF0D7
:10216000AD6B01DC020E996FFDEC0BF08C2BF1D7FF
:102170008B2BEBD711EC0CF01E6A0C0E1D6E1C6A3B
:102180001B6A226A180E216E206A1F6A266A300EA8
:10219000256E246A236A2A6A600E296E286A276AD5
:1021A0002E6AC00E2D6E2C6A2B6A010E326E800EC6
:1021B000316E306A2F6A030E366E356A346A336ABE
:1021C000070E3A6E39683868F80E376E070E3E6EA5
:1021D0003D683C68F80E3B6E030E426E416A406AF1
:1021E0003F6A010E466E800E456E446A436A4A6A33
:1021F000C00E496E486A476A4E6A600E4D6E4C6A60
:102200004B6A526A300E516E506A4F6A566A180E07
:10221000556E546A536A5A6A0C0E596E586A576A58
:102220008E6B8D6B8E53D8A48AD08D513108D8A077
:1022300086D08B6B8B510F08D8A079D08B51040DB1
:10224000F3509A6B996F1B0E9925E96E000E9A2137
:10225000EA6EEFCF9BF0ECCF9CF0ECCF9DF0ECCF93
:102260009EF0006A016A026A9E51800B036E005262
:1022700006E1015204E1025202E1035203E0010EC1
:102280008C6F01D08C6B8B51040DF3509A6B996F4E
:102290001B0E9925016E000E9A2101C09BF09C6FC8
:1022A0008B51040DF3509E6B9D6F1B0E9D25E96EA7
:1022B000000E9E21EA6EEFCF9FF0ECCFA0F0ECCFA6
:1022C000A1F0ECCFA2F0D8909F35006EA035016E42
:1022D000A135026EA2359CC0EAFF9BC0E9FF00C099
:1022E000EFFF01C0ECFF02C0ECFFEC6E8C531DE071
:1022F0008B51040DF3509A6B996F1B0E9925E96E63
:10230000000E9A21EA6EEF500109ECCF01F0ECCFFC
:1023100002F0ECCF03F0ED52ED52ED52EF6E01C042
:10232000ECFF02C0ECFF03C0ECFF8B2B83D7190E30
:10233000996FFDEC0BF08D2BD8B48E2B73D788EFF3
:1023400018F0050E006E002EFED7120092948984BC
:10235000F8DF929689969296F4DF92948994F1DF51
:1023600012009286EEDF92948984EBDF9294899436
:102370001200929689969296E4DF92948984E1DF26
:1023800092948994120092AF02D0EBDF01D0F1DF7A
:1023900092AD02D0E6DF01D0ECDF92AB02D0E1DFFC
:1023A00001D0E7DF92A902D0DCDF01D0E2DF92A703
:1023B00002D0D7DF01D0DDDF92A502D0D2DF01D07D
:1023C000D8DF92A302D0CDDF01D0D3DF92A102D01B
:1023D000C8DF01D0CEDF1200916B9286B2DF9294FB
:1023E0008984AFDF928680A607D0ABDF912B915115
:1023F0000A08D8B401D0F6D792948994A2DF9296B5
:10240000899692969EDF91510A0804E1010E016EB1
:1024100003D002D0000E016E1200928692DF9294D9
:1024200089848FDF9296899692968BDF9294899415
:1024300088DF56EF12F08F6B92868E6B8E510708F5
:102440000EE3D8908F37929489847BDF928680A6A2
:1024500001D08F819294899474DF8E2BEFD78FC037
:1024600001F012008C6B9296899692966ADF929494
:10247000898467DF9294899464DF928662DF000E1C
:10248000016E70EF12F09296899692965ADF9294AE
:10249000898457DF928655DF120058DFD00E926F85
:1024A00072DF9ADF926B6FDF97DFB7D7D10E926F33
:1024B0006ADF92DF8B6B8B51050814E3036A8B5143
:1024C000730F016E000E032201C08CF003C08DF06B
:1024D000B2DF8DC0EAFF8CC0E9FF01C0EFFFC2D7B9
:1024E0008B2BE9D7036A8B51730F016E000E032209
:1024F00001C08CF003C08DF09EDF8DC0EAFF8CC060
:10250000E9FF01C0EFFF68DFBEDF7939006E0F0E13
:10251000001600500A0DF3CF6CF079510F0B6C27A9
:1025200078A903D00A0E6D6F01D06D6B78510F0B37
:102530006D277739006E0F0E001600500A0DF3CF8D
:102540006EF077510F0B6E277651070B6F6F753951
:10255000006E0F0E001600500A0DF3CF71F075518A
:102560000F0B71277439006E0F0E001600500A0D04
:10257000F3CF70F074510F0B70277339006E0F0E8C
:10258000001600500A0DF3CF72F073510F0B722733
:102590002AEF18F09F51016A9E5D03E29EC000F091
:1025A0000CD0006A080EA06F9E3700369F51005C69
:1025B000D8B0006E0136A02FF7D71200200E99A9CF
:1025C000300E9A6F98C000F098AF08D0001E002A15
:1025D00000C098F02D0E9A6F998F9981015098C084
:1025E0009EF0640E9F6FD6DF00C098F0300E01247D
:1025F0009B6F98C09EF00A0E9F6FCCDF300E0024B8
:102600009D6F300E01249C6F9AC000F0300E9B5DD0
:1026100004E0998399BF998512D09AC09BF0200E4F
:102620009A6F300E9C5D04E0998199BF998307D021
:10263000D8A4998104E19BC09CF0200E9B6F99B5B2
:1026400005D099B307D099B109D00CD09AC0A4F0A5
:102650002CEC0CF09BC0A4F02CEC0CF09CC0A4F073
:102660002CEC0CF09DC0A4F02CEC0CF012006D5181
:10267000010A1CE0030A27E0010A32E0070A3DE0F4
:10268000010A48E0030A53E0010A5EE00F0AD8B4E9
:1026900068D0010AD8B472D0030AD8B47CD0010A39
:1026A000D8B486D0070AD8B490D09CD0EA6A8B0EF2
:1026B000E96E000EF2EC08F00A000900F550EE6E2B
:1026C0000009FBE18FD0EA6A8B0EE96E000EFCEC8C
:1026D00008F00A000900F550EE6E0009FBE182D017
:1026E000EA6A8B0EE96E000E06EC09F00A0009009A
:1026F000F550EE6E0009FBE175D0EA6A8B0EE96ECB
:10270000000E10EC09F00A000900F550EE6E000909
:10271000FBE168D0EA6A8B0EE96E000E1AEC09F054
:102720000A000900F550EE6E0009FBE15BD0EA6A91
:102730008B0EE96E000E24EC09F00A000900F5503A
:10274000EE6E0009FBE14ED0EA6A8B0EE96E000ED8
:102750002EEC09F00A000900F550EE6E0009FBE1CD
:1027600041D0EA6A8B0EE96E000E38EC09F00A00DF
:102770000900F550EE6E0009FBE134D0EA6A8B0ED9
:10278000E96E000E42EC09F00A000900F550EE6E09
:102790000009FBE127D0EA6A8B0EE96E000E4CECD3
:1027A00009F00A000900F550EE6E0009FBE11AD0AD
:1027B000EA6A8B0EE96E000E56EC09F00A00090079
:1027C000F550EE6E0009FBE10DD0EA6A8B0EE96E62
:1027D000000E60EC09F00A000900F550EE6E0009E9
:1027E000FBE100D0996B9A6B9C6B8B0E9B6F9EEC00
:1027F0000EF07B6B8B0E7A6F6EC098F0110E996F96
:10280000DDDE120E996F9A6B9C6B8B0E9B6F9EECAC
:102810000EF07B6B8B0E7A6F71C098F0110E996F72
:10282000CDDE996B080E9A6F9C6B8B0E9B6F9EECA6
:102830000EF07B6B8B0E7A6F3A0EA46F2CEC0CF0C3
:102840000C0E996F080E9A6F9C6B8B0E9B6F9EEC13
:102850000EF07B6B8B0E7A6F70C098F0110E996F33
:10286000ADDE8B51200802E1300E8B6F110E996F97
:10287000080E9A6F9C6B8B0E9B6F9EEC0EF0725144
:102880001D080FE21E0EAB6FAC6B010EAD6FB3EC0B
:102890000CF01F0EAB6FAC6B010EAD6FB3EC0CF018
:1028A0000CD01E0EAB6FAC6BAD6BB3EC0CF01F0E0F
:1028B000AB6FAC6BAD6BB3EC0CF072C09EF01E0E48
:1028C0009F6F68DE00C095F095511C0808E21E0E4F
:1028D000AB6F010EAC6FAD6FB3EC0CF007D01E0EFA
:1028E000AB6F010EAC6FAD6BB3EC0CF01C0E966FC2
:1028F000020E976F9651955D09E31F0EAB6F97C05F
:10290000ACF0010EAD6FB3EC0CF007D01F0EAB6F47
:1029100097C0ACF0AD6BB3EC0CF096079651955D9B
:1029200009E31E0EAB6F97C0ACF0010EAD6FB3ECB8
:102930000CF007D01E0EAB6F97C0ACF0AD6BB3ECD4
:102940000CF09607972B9653D5E12CEF18F0090061
:10295000F5520DE0F6CF95F0F7CF96F0F5CFA4F055
:102960002CEC0CF095C0F6FF96C0F7FFF0D71200E4
:1029700011EC0CF07B6B8B0E7A6F960EF66E170EC9
:10298000F76EE5DF996B9A6B9C6B8B0E9B6F9EECE1
:102990000EF07B6B8B0E7A6F9C0EF66E170EF76E39
:1029A000D6DF996B080E9A6F9C6B8B0E9B6F9EEC1B
:1029B0000EF0938A81AA02D0938881A8FAD7666B19
:1029C00066C05EF0676B67C05FF011EC0CF07B6B6C
:1029D0008B0E7A6FA20EF66E170EF76EB8DF996B3C
:1029E0009A6B9C6B8B0E9B6F9EEC0EF0D00E6C2541
:1029F000956F070E966FD8B0962B7B6B8B0E7A6F08
:102A0000020EE96E96C09CF095C09BF03AEC0CF07B
:102A1000996B080E9A6F9C6B8B0E9B6FCCEC0DF034
:102A20005F5206E05F6A6C2B6C51640801E16C6BCD
:102A30005E52DCE05E6A7B6B8B0E7A6FA80EF66EE0
:102A4000170EF76E84DF996B9A6B9C6B8B0E9B6FE6
:102A50009EEC0EF06D51010A1CE0030A27E0010A0A
:102A600032E0070A3DE0010A48E0030A53E0010AA8
:102A70005EE00F0AD8B468D0010AD8B472D0030A55
:102A8000D8B47CD0010AD8B486D0070AD8B490D084
:102A90009CD0EA6A8B0EE96E000E6AEC09F00A001F
:102AA0000900F550EE6E0009FBE18FD0EA6A8B0E4B
:102AB000E96E000E75EC09F00A000900F550EE6EA3
:102AC0000009FBE182D0EA6A8B0EE96E000E80EC11
:102AD00009F00A000900F550EE6E0009FBE175D01F
:102AE000EA6A8B0EE96E000E8BEC09F00A00090011
:102AF000F550EE6E0009FBE168D0EA6A8B0EE96ED4
:102B0000000E96EC09F00A000900F550EE6E00097F
:102B1000FBE15BD0EA6A8B0EE96E000EA1EC09F0D6
:102B20000A000900F550EE6E0009FBE14ED0EA6A9A
:102B30008B0EE96E000EACEC09F00A000900F550AE
:102B4000EE6E0009FBE141D0EA6A8B0EE96E000EE1
:102B5000B7EC09F00A000900F550EE6E0009FBE140
:102B600034D0EA6A8B0EE96E000EC2EC09F00A005E
:102B70000900F550EE6E0009FBE127D0EA6A8B0EE2
:102B8000E96E000ECDEC09F00A000900F550EE6E7A
:102B90000009FBE11AD0EA6A8B0EE96E000ED8EC50
:102BA00009F00A000900F550EE6E0009FBE10DD0B6
:102BB000EA6A8B0EE96E000EE3EC09F00A000900E8
:102BC000F550EE6E0009FBE100D0996B080E9A6F8C
:102BD0009C6B8B0E9B6FCCEC0DF05F5207E05F6A35
:102BE0006D2B6D510D0802E1010E6D6F5E52D8B470
:102BF00031D75E6A7B6B8B0E7A6FAE0EF66E170E58
:102C0000F76EA5DE996B9A6B9C6B8B0E9B6F9EEC9F
:102C10000EF07B6B8B0E7A6F6EC098F0110E996F71
:102C2000CDDC200EA46F2CEC0CF0200EA46F2CEC4D
:102C30000CF0996B080E9A6F9C6B8B0E9B6FCCEC13
:102C40000DF05F5207E05F6A6E2B6E51200802E1C3
:102C5000010E6D6F5E52DDE05E6A7B6B8B0E7A6FEC
:102C6000B40EF66E170EF76E72DE996B9A6B9C6B54
:102C70008B0E9B6F9EEC0EF06F51010A0DE0030A64
:102C800018E0010A23E0070A2EE0010A39E0030AEE
:102C900044E0010A4FE05BD0EA6A8B0EE96E000E59
:102CA000EEEC09F00A000900F550EE6E0009FBE1B8
:102CB0004ED0EA6A8B0EE96E000EF9EC09F00A00BC
:102CC0000900F550EE6E0009FBE141D0EA6A8B0E77
:102CD000E96E000E04EC0AF00A000900F550EE6EF1
:102CE0000009FBE134D0EA6A8B0EE96E000E0FECAE
:102CF0000AF00A000900F550EE6E0009FBE127D04A
:102D0000EA6A8B0EE96E000E1AEC0AF00A0009005E
:102D1000F550EE6E0009FBE11AD0EA6A8B0EE96EFF
:102D2000000E25EC0AF00A000900F550EE6E0009CD
:102D3000FBE10DD0EA6A8B0EE96E000E30EC0AF072
:102D40000A000900F550EE6E0009FBE100D0996B16
:102D5000080E9A6F9C6B8B0E9B6FCCEC0DF05F5244
:102D600007E05F6A6F2B6F51080802E1010E6F6F79
:102D70005E5282E05E6A7B6B8B0E7A6FBA0EF66EE5
:102D8000170EF76EE4DD996B9A6B9C6B8B0E9B6F45
:102D90009EEC0EF07B6B8B0E7A6F71C098F0110E6B
:102DA000996F0CDC200EA46F2CEC0CF0200EA46F9D
:102DB0002CEC0CF0996B080E9A6F9C6B8B0E9B6F32
:102DC000CCEC0DF05F5206E05F6A712B7151180870
:102DD00001E1716B5E52DEE05E6A7B6B8B0E7A6F97
:102DE000C00EF66E170EF76EB2DD996B9A6B9C6B88
:102DF0008B0E9B6F9EEC0EF07B6B8B0E7A6F70C010
:102E000098F0110E996FDEEC12F0200EA46F2CECEE
:102E10000CF0200EA46F2CEC0CF0996B080E9A6F3E
:102E20009C6B8B0E9B6FCCEC0DF05F5206E05F6AE3
:102E3000702B70513C0801E1706B5E52DDE05E6A00
:102E40007B6B8B0E7A6FC60EF66E170EF76E7FDDFC
:102E5000996B9A6B9C6B8B0E9B6F9EEC0EF07B6B51
:102E60008B0E7A6F200EA46F2CEC0CF072C098F0D1
:102E7000110E996FDEEC12F0200EA46F2CEC0CF00A
:102E8000996B080E9A6F9C6B8B0E9B6FCCEC0DF0C0
:102E90005F5206E05F6A702B72513C0801E1726B71
:102EA0005E52DDE05E6A32EF18F08DC019F01A6AEA
:102EB000A6EC11F08D51FE0B916F926FC3EC11F0E7
:102EC000ECEC11F0015206E043EC12F0010E1A6E28
:102ED000016E22D08EC092F0C3EC11F0ECEC11F038
:102EE000015207E043EC12F0020E1A6E010E016E61
:102EF00013D08FC092F0C3EC11F0ECEC11F0015242
:102F000007E043EC12F0030E1A6E010E016E04D0BE
:102F100043EC12F0000E016E13EF18F072C09EF039
:102F20000A0E9F6FCAEC12F001388C6FF00E8C17EE
:102F300072C09EF00A0E9F6FCAEC12F000508C1106
:102F4000736F70C09EF00A0E9F6FCAEC12F00138CA
:102F50008C6FF00E8C1770C09EF00A0E9F6FCAEC3B
:102F600012F000508C11746F71C09EF00A0E9F6FAA
:102F7000CAEC12F001388C6FF00E8C1771C09EF005
:102F80000A0E9F6FCAEC12F000508C11756F6FC063
:102F900076F06EC09EF00A0E9F6FCAEC12F00138F8
:102FA0008C6FF00E8C176EC09EF00A0E9F6FCAECED
:102FB00012F000508C11776F6DC09EF00A0E9F6F5B
:102FC000CAEC12F001388C6FF00E8C176DC09EF0B9
:102FD0000A0E9F6FCAEC12F000508C11786F6CC013
:102FE0009EF00A0E9F6FCAEC12F001388C6FF00E43
:102FF0008C176CC09EF00A0E9F6FCAEC12F0005046
:103000008C11796F070E8B6F8B07036A8B51730FCF
:10301000E96E000E0320EA6EEFCF8FF0D00E8D6FB9
:103020008BC08EF042D78B53EFE1120072511D0816
:1030300002E3726B0BD0726B702B70513C0806E18F
:10304000706B712B7151180801E1716B3BEF18F037
:103050004DEF12F037EF13F0665307E05E6A5EC083
:1030600066F086D45BDF11EC0CF05F5207E05F6A1C
:103070005FC067F0DBD752DF11EC0CF08CEF18F07B
:10308000F86AD09E078E700ED36E9B8C9B9E5B6AF7
:10309000696B686B6A6B6B6B7B6B7A6B0F01386B60
:1030A000396B3A6B776A786A796A010E5C6E5D6E8D
:1030B0005E6A5F6A0001606B616B626B636B646B7D
:1030C000656B666B676B700ED36E9B8C9B9EE6EF99
:1030D0000BF0F5EF0BF0300E616EF19E010E996F63
:1030E000FDEC0BF0938A81BA03D0010E8A6F01D0F8
:1030F0008A6B640E996FFDEC0BF09496C30ED56E3F
:10310000F28AC00EF21211EC0CF05B6A8A5304E0F2
:0E31100029EF10F0FDD702D09BD7FED70300A9
:020000040030CA
:0E00000000E8183C003F81000FC00FE00F40E9
:00000001FF
